:020000041800E2
:1040000000800020AD400018D3400018D5400018B3
:1040100000000000000000000000000000000000A0
:10402000000000000000000000000000D740001861
:104030000000000000000000D9400018DB4000181C
:10404000D1410018DD400018DD400018DD400018A7
:10405000DD400018DD400018DD400018DD4000188C
:10406000DD400018DD400018DD400018DD4000187C
:10407000DD400018DD400018DD400018DD4000186C
:10408000DD400018DD400018DD400018DD4000185C
:10409000DD400018DD4000180348854600F064F854
:1040A000004800472D4600180080002000200C49E1
:1040B00008600C480C49086001200C4908600C4855
:1040C0000C4988470C480D4908600D4988470D4840
:1040D0000047FEE7FEE7FEE7FEE7FEE7FEE700003B
:1040E0002C100040254000180C0000190000001999
:1040F0000040001831450018944801005410034056
:104100005546001899400018F0B51FB40646002027
:1041100082B005464024019100901BE0019922469F
:104120000F46304600F042F8049A059B801A9941E8
:1041300010D310461946224600F028F8361A8F414F
:104140000197224601200021009F00F01FF8381837
:104150004D4100902046641E0028DFDC019B009842
:104160002946324607B0F0BD064C0125064E05E053
:10417000E36807CC2B430C3C98471034B442F7D388
:10418000FFF78EFF084800182848001810B5202AAD
:1041900004DB0146203A9140002010BD91402023CD
:1041A0009C1A0346E3401943904010BD10B5202AE5
:1041B00004DB0846203AD040002110BD0B46D34016
:1041C000D0402024A21A91400843194610BD000097
:1041D00070B50D4AD0680D4900230B7001260C4CB8
:1041E00093142360850504D5551555610D78354325
:1041F0000D70400506D5012080025061087802222A
:1042000010430870636070BD008002409C30002045
:10421000000001400FB410B503A9044B044A0298F2
:1042200000F018F810BC08BC04B018471D46001870
:104230009830002002E008C8121F08C1002AFAD1F5
:1042400070477047002001E001C1121F002AFBD116
:1042500070470000FFB58FB00F460446002606E009
:1042600025280AD0129A11999047641C761C207850
:104270000028F5D1304613B0F0BD00250121A14A38
:10428000009500E00543641C23780846203B9840D5
:104290001042F7D120782E2815D1042005436078EC
:1042A000641C2A280AD101CF641C00900BE00099FD
:1042B0000A22514330394018641C0090207801468E
:1042C00030390929F3D920786C280ED004DC4C2829
:1042D00013D06A2812D104E074280ED07A280DD1A8
:1042E0000BE001204005054307E001210905627844
:1042F0000D43824201D16D18641C641C20788646EF
:1043000069284AD008DC0028B4D058286DD063282A
:1043100010D0642808D140E070286BD0732812D0E8
:10432000752860D0782860D0129A7046119990470D
:10433000761CE5E03878694608720020487202A8C9
:104340000190012003E0386801900020C0433F1D28
:1043500069070CD5002500E06D1C00998D420FDA2D
:104360008542F9DB0199495D0029F5D108E0002576
:1043700000E06D1C8542FCDB0199495D0029F8D104
:10438000761907E0019801990078491C0191129A69
:10439000119990476D1EF5D2B2E00A2002900021DB
:1043A0006802400F039102280CD001CFC117844648
:1043B00000290DDA624608465242002181419446A6
:1043C0002D2008E0FF1DFF08FF0003CF8446EFE724
:1043D000280504D52B206A46107401203CE0E8072C
:1043E0003AD02020F7E70A2000E0102000210391B6
:1043F000029007E0102002900021042005430820CD
:10440000039100906802400F022810D001CF0021D4
:10441000844600200D9028071FD5704670280CD0C8
:10442000029A1020039B42401A430CD015E0FF1D56
:10443000FF08FF0003CF8446EBE740206A46107474
:1044400001200D900CE06046084306D030206A46FB
:1044500010747046507402200D907046582804D095
:1044600029A001900DA80E900DE02CA0F9E7604660
:10447000039B029AFFF748FE019B84469B5C0E9AC1
:10448000521E0E92137060460843F0D10E9805A993
:10449000081A20300190680701D5009801E001203A
:1044A00000900199884203DD01460198081A00E056
:1044B00000200025009006E004A8129A405D1199A2
:1044C00090476D1C761C0D988542F5DB04E0129A2E
:1044D000302011999047761C0099481E00900029C1
:1044E000F5DC08E00E980E990078491C0E91129A9E
:1044F00011999047761C0199481E01900029F1DC22
:10450000641CB4E6092801003031323334353637C3
:10451000383961626364656600000000303132330F
:1045200034353637383941424344454600000000AF
:1045300010B5084B00218A008458D2181460491C19
:104540002629F8D3BFF35F8F03488360BFF34F8FF3
:1045500010BD00000030002000ED00E010B5072283
:104560000621002000F00EF903228B21002000F02C
:10457000F1F810BD01241449200348600862FF20AF
:10458000124981300860091D0860114800F02CF8BC
:1045900003256D022946072000F038F829460A2035
:1045A00000F034F82946002000F030F809480025D2
:1045B000046062B6084C20780028FCD0217807A05F
:1045C000FFF728FE2570F6E7000001402421004097
:1045D000040F000000E100E09C3000205472696785
:1045E0003A2025580D0A000001218907CB6A8A1557
:1045F0001343CB624B6A13434B624B6A93434B6248
:104600000149C8627047000000800240024A8000F1
:1046100080180160704700000080024010B5044619
:10462000C1B2002000F0E6F8204610BD0449002089
:104630008847FFF793FF03A0FFF7ECFDFFF79AFF12
:10464000D10800004558544920546573742E2E2E0D
:104650000D0A0000F0B5364C87B0A06881B235482D
:104660000818A060354D3448E8633549102088604B
:10467000344FB8693449884257D16E46002001A9A9
:104680008200D3191B68401CB3500628F8D3086970
:104690000A22431C002B25D01346834322D1A36852
:1046A0001F263605C005C00EB34300050343A360B3
:1046B000E86B0B8A400940019B04DB0E1843E8635A
:1046C000A0680E690F231B04B603360F9843360407
:1046D0003043A060E86B98430B699B021B0F1B04DF
:1046E0001843E863C868194B441C05D0144684433A
:1046F00002D18005800E18610868441C08D08243EE
:1047000006D15A69800592099201800E02435A61CE
:104710008868411C09D0002807D00D4BD9697C223C
:10472000800A914310400143D96107B0F0BD0000F9
:10473000000003400000B1011403740000100340A6
:1047400000100040000F0018B6D5F5C84010034017
:1047500040C002400A4B000310B5C0180023C360DC
:10476000C36880242343C3608160C168A143C160E2
:10477000C16907231943C16120210A43C26010BDEA
:104780000030024030B5FF24174B82349500ED18FD
:104790002C60A1248900CB181C6043008024134D99
:1047A000234349190B60114621430F4CC300803C41
:1047B0001B195960E105CC6A0123C01C83401C43CE
:1047C000CC62486A18434862486A984348620920A4
:1047D000074B03E05969D140C90704D10146401E87
:1047E000C0B20029F6D130BD0021004000200040B9
:1047F00000000140034A00038018026A9206FCD5BB
:10480000416070470030024028480018983000206E
:1048100004000000344200182C4800189C3000208E
:0C482000040000004442001800000000EA
:040000051800409906
:00000001FF
